:020000040000FA
:100000000FEF00F00000FFFF78EF00F0FFFFFFFFB1
:10001000FFFFFFFFFFFFFFFF0000A1EF00F098ECE4
:1000200001F0096A0B6A0A6A056A066A6FEC01F058
:100030007EEC01F09BEC01F0A2EC01F0D4EC01F0BD
:10004000AFEC01F0066A1B6A1E6A06826C949E90F1
:10005000A9EC01F0C4CF1DF0C4CF0BF0C4CF22F047
:10006000C4CF23F0080E096EC2822EEC01F0BDEC65
:1000700000F06CB461EC01F0C80E1E6046EF00F0B9
:10008000080E1B606AEF01F048EF00F005921B6A52
:100090009EA06DEF00F00B0ECF6EDB0ECE6E9E902D
:1000A0001E2A05A21E6A0B50096061EF00F009507C
:1000B0000B5C0208D8B06BEF00F0020E09266DEF62
:1000C00000F00B50095C0408D8B06BEF00F0040E90
:1000D000095E6DEF00F00BC009F0000E095CD8A4BA
:1000E00075EF00F06B6A8098C4D76B688098C1D7B1
:1000F000F2B48DEF00F021A0110011C079FF12C001
:1001000078FF13C077FF14C076FF15C075FF16C0C7
:1001100074FF2190A498F28E1100F29E07C0D7FFC1
:1001200008C0D6FF9EAC9AEF00F0A2EC00F0C282AD
:100130002EEC01F027EC01F0BDEC00F0F294F28E11
:1001400011001100C4CF1DF0C4CF0BF0C4CF22F0BA
:10015000C4CF23F02232229E070E0B640B6EF00EEA
:100160000B600B6ED8901D32D8901D32D8901D3286
:1001700082B00B6A068C9E9C1200800E222409021B
:10018000D890F336F436F4CF1CF0F00ED8B01C6ED5
:10019000F00E1C601C6E1C50FF081D02F4CFE8FF1F
:1001A0001C26D8B01C68F00E1C601C6E0050EB5072
:1001B0001C02F4CF12F0F3CF11F00050280FEB50D7
:1001C0001C02F4CF14F0F3CF13F00050500FEB509B
:1001D0001C02F4CF16F0F3CF15F0D8901232113282
:1001E00012321132123211321232113212321132F3
:1001F0000F0E1216D89014321332143213321432F6
:10020000133214321332143213320F0E1416D890E4
:1002100016321532163215321632153216321532A2
:10022000163215320F0E1616F00E1126D8B0122AFD
:10023000F00E1326D8B0142AF00E1526D8B0162AC0
:10024000FC0EFC0EFC0E21806E92069C1200230E0A
:10025000006002D0002A1200006A1200069C11EE13
:1002600000F009C0E8FF020DF3CFE1FFF4CFE8FF93
:10027000E226E6CF08F0E6CF07F012009D9CF29A46
:100280006B6A006A059012000B6A0A6A06889D8CE8
:10029000AFEC01F0BDEC00F027EC01F0F28AFF0EAC
:1002A0006B6E120082B05BEF01F006B2120044ECFC
:1002B00001F00682120006A212003EEC01F0069246
:1002C00012006CA469EF01F0096A05821B2A6C9484
:1002D000120012006B6A82B0FF006AEF01F0100E8C
:1002E000C16E360EC06E400E9A6E000E996E0F0EE5
:1002F000B86E0F0E926E150EC26E1200000E7F6E5B
:10030000800E7E6EF30E7B6E010E7A6E400E6F6E67
:10031000010E6E6E4F0E6D6EFF0E6B6E000E6A6EEE
:10032000830E6C6E000E716E000E706E7E8E12006B
:10033000FF0E946E1200800ED56EF80ED76E5E0E14
:10034000D66E1200B10ECD6E0B0ECF6EDB0ECE6EE2
:100350001200F28A130ED06EF28EA3881200006A89
:10036000000E096E0B6EFD0E076ED76E2C0ED66E4C
:10037000086E600EE96E000EEA6E82A6CAEF01F00A
:10038000880EE16E000EE26EB00ED96E000EDA6ECF
:1003900005801200880ED96E000EDA6EB00EE16E86
:1003A000000EE26E05801200000EF86E060EF76E6B
:1003B000000EF66E00EE60F0270E0C6E0900F5CF11
:1003C000EEFF0C2EFBD700EE60F0000EF86E060E6E
:1003D000F76E280EF66E280EE926270E0C6E090021
:1003E000F5CFEEFF0C2EFBD700EE60F0000EF86E9E
:1003F000060EF76E500EF66E500EE926270E0C6EA6
:100400000900F5CFEEFF0C2EFBD700EE60F0000EDA
:10041000F86E060EF76E780EF66E11EE00F0FF0E17
:100420000C6E0900F5CFE6FF0C2EFBD70900F5CFC7
:10043000E6FF11EE00F0000EF86E070EF76E780E74
:10044000F66E12EE00F0FF0E0C6E0900F5CFE6FF1F
:100450000C2EFBD70900F5CFE6FF12EE00F01200DC
:10046000FFFFFFFFFFFFFFFFFFFFFFFFFFFFFFFF9C
:10047000FFFFFFFFFFFFFFFFFFFFFFFFFFFFFFFF8C
:10048000FFFFFFFFFFFFFFFFFFFFFFFFFFFFFFFF7C
:10049000FFFFFFFFFFFFFFFFFFFFFFFFFFFFFFFF6C
:1004A000FFFFFFFFFFFFFFFFFFFFFFFFFFFFFFFF5C
:1004B000FFFFFFFFFFFFFFFFFFFFFFFFFFFFFFFF4C
:1004C000FFFFFFFFFFFFFFFFFFFFFFFFFFFFFFFF3C
:1004D000FFFFFFFFFFFFFFFFFFFFFFFFFFFFFFFF2C
:1004E000FFFFFFFFFFFFFFFFFFFFFFFFFFFFFFFF1C
:1004F000FFFFFFFFFFFFFFFFFFFFFFFFFFFFFFFF0C
:10050000FFFFFFFFFFFFFFFFFFFFFFFFFFFFFFFFFB
:10051000FFFFFFFFFFFFFFFFFFFFFFFFFFFFFFFFEB
:10052000FFFFFFFFFFFFFFFFFFFFFFFFFFFFFFFFDB
:10053000FFFFFFFFFFFFFFFFFFFFFFFFFFFFFFFFCB
:10054000FFFFFFFFFFFFFFFFFFFFFFFFFFFFFFFFBB
:10055000FFFFFFFFFFFFFFFFFFFFFFFFFFFFFFFFAB
:10056000FFFFFFFFFFFFFFFFFFFFFFFFFFFFFFFF9B
:10057000FFFFFFFFFFFFFFFFFFFFFFFFFFFFFFFF8B
:10058000FFFFFFFFFFFFFFFFFFFFFFFFFFFFFFFF7B
:10059000FFFFFFFFFFFFFFFFFFFFFFFFFFFFFFFF6B
:1005A000FFFFFFFFFFFFFFFFFFFFFFFFFFFFFFFF5B
:1005B000FFFFFFFFFFFFFFFFFFFFFFFFFFFFFFFF4B
:1005C000FFFFFFFFFFFFFFFFFFFFFFFFFFFFFFFF3B
:1005D000FFFFFFFFFFFFFFFFFFFFFFFFFFFFFFFF2B
:1005E000FFFFFFFFFFFFFFFFFFFFFFFFFFFFFFFF1B
:1005F000FFFFFFFFFFFFFFFFFFFFFFFFFFFFFFFF0B
:1006000075899CAFBFCEDAE2E8EAE8E2DACEBFAFA6
:100610009C8975604D3A2A1B0F07010001070F1BCB
:100620002A3A4D6000000000DACEBFAF9C897560A9
:100630004D3A2A1B0F07010001070F1B2A3A4D6094
:1006400075899CAFBFCEDAE2E8EAE8E2000000007C
:100650000F07010001070F1B2A3A4D6075899CAFF7
:10066000BFCEDAE2E8EAE8E2DACEBFAF9C89756095
:100670004D3A2A1B00000000739373937393739396
:10068000739373937393F5A296AEA2B7DEBECAC4FA
:10069000B9C9E6CD7AD194D44BD7B0D9D1DBB8DD86
:1006A0006FDFFCE065E2AEE3DCE4F2E5F3E6E0E711
:1006B000BDE88AE94AEAFDEAA5EB43ECD8EC64ED33
:1006C000E8ED65EEDCEE4CEFB7EF1DF07EF0DAF012
:1006D00032F186F1D7F124F26EF2B5F2F9F23AF383
:1006E00079F3B6F3F0F328F45EF492F4C5F4F6F47B
:1006F00025F552F57EF5A9F5D2F5FAF521F647F67E
:100700006CF68FF6B2F6D3F6F4F613F732F750F72D
:100710006EF78AF7A6F7C1F7DBF7F5F70EF827F8BB
:100720003FF856F86DF883F899F8AEF8C3F8D7F8A3
:10073000EBF8FFF812F924F937F949F95AF96BF98E
:100740007CF98DF99DF9ADF9BCF9CCF9DBF9E9F942
:10075000F8F906FA14FA21FA2FFA3CFA49FA56FA8D
:1007600062FA6EFA7BFA86FA92FA9EFAA9FAB4FA5B
:10077000BFFACAFAD4FADFFAE9FAF3FAFDFA07FB8C
:1007800010FB1AFB23FB2CFB36FB3EFB47FB50FB0D
:1007900059FB61FB69FB72FB7AFB82FB89FB91FBD6
:1007A00099FBA0FBA8FBAFFBB7FBBEFBC5FBCCFBDB
:1007B000D3FBDAFBE0FBE7FBEDFBF4FBFAFB01FC10
:1007C00007FC0DFC13FC19FC1FFC25FC2BFC30FC6A
:1007D00036FC3CFC41FC47FC4CFC52FC57FC5CFCEE
:1007E00061FC66FC6BFC70FC75FC7AFC7FFC84FC95
:1007F00089FC8DFC92FC97FC9BFCA0FCA4FCA8FC53
:10080000ADFCB1FCB5FCBAFCBEFCC2FCC6FCCAFC2B
:10081000CEFCD2FCD6FCDAFCDEFCE2FCE6FCE9FC19
:10082000EDFCF1FCF4FCF8FCFCFCFFFC03FD06FD18
:100830000AFD0DFD10FD14FD17FD1AFD1EFD21FD25
:1008400024FD27FD2BFD2EFD31FD34FD37FD3AFD46
:100850003DFD40FD43FD46FD49FD4CFD4FFD51FD75
:1008600054FD57FD5AFD5CFD5FFD62FD65FD67FDB2
:100870006AFD6CFD6FFD72FDFFFFFFFFFFFFFFFFD5
:10088000FFFFFFFFFFFFFFFFFFFFFFFFFFFFFFFF78
:10089000FFFFFFFFFFFFFFFFFFFFFFFFFFFFFFFF68
:1008A000FFFFFFFFFFFFFFFFFFFFFFFFFFFFFFFF58
:1008B000FFFFFFFFFFFFFFFFFFFFFFFFFFFFFFFF48
:020000040030CA
:0E00000000060E3E381D81000C000FE00F4080
:020000040020DA
:08000000FFFFFFFFFFFFFFFF00
:00000001FF
